:100000000C942A000C9434000C9434000C943400AA
:100010000C9434000C9434000C9434000C94340090
:100020000C9434000C9434000C9434000C94340080
:100030000C9434000C9434000C9434000C94340070
:100040000C9434000C9434000C9434000C94340060
:100050000C94340011241FBECFE5D4E0DEBFCDBF29
:100060000E9436000C9445000C94000010BC85E002
:1000700089B988E18AB986E880BD8FEF8ABB1BBA4F
:0E0080005F9BFECF8CB18BBBFBCFF894FFCF04
:00000001FF
